S12380000F8690B710398E00FF8630B710308640B710248608B710268602B710098620B71C
S1238020102B862CB7102DB6102F7F000B7F000C0ECE08E0C60218CE0019BD8051BD807784
S1238040960C2703BD81AF7E803DDF09DE0926FC3918DF03BD82D018DE0318DF0718DE0701
S123806026FB7F10227F102018DE0318DF0718DE0726FB5A26DE39960B81FF27037E812A5B
S12380807F000B7F000CBD82A896008141273E8161273A81422748816227448143274E81A6
S12380A063274A8144275881642754815227628172275E8153275E8173275A813025098142
S12380C0372205BD812B2062BD814B205DCE8462BD82C3F610004FBD8263BD82A8204B7FCF
S12380E01004CE8477BD82C3BD82A8203DCE8469BD82C3F610034FBD8263BD82A8202BCEA2
S12381008470BD82C3F610084FBD8263BD82A82019970C2015CE8486BD82C3BD82A8CE08D7
S1238120E0C60218CE0019BD805139C60180302704584A26FCF510042703532007FA1004AC
S1238140F7100439F41004F7100439BD82B3CE8410BD82C3BD82A8CE83E9BD82C3BD82A82B
S1238160CE8410BD82C3BD82A8CE8310BD82C3BD82A8CE8329BD82C3BD82A8CE8344BD822F
S1238180C3BD82A8CE835DBD82C3BD82A8CE8376BD82C3BD82A8CE8399BD82C3BD82A8CE49
S12381A083BDBD82C3BD82B3CE83E7BD82C3398630B71030CE843ABD82C3F610314FBD8214
S12381C0638620BD829FCE843FBD82C3F610324FBD82638620BD829FCE8444BD82C3F610D6
S12381E0334FBD82638620BD829FCE8449BD82C3F610344FBD82638620BD829F8634B71006
S123820030CE844EBD82C3F610314FBD82638620BD829FCE8453BD82C3F610324FBD82630C
S12382208620BD829FCE8458BD82C3F610334FBD82638620BD829FCE845DBD82C3F6103471
S12382404FBD8263860DBD829F394FCE0064028FD7018FCE000A02D7028F58585858DA0288
S1238260D702394FBD824A96018B30BD829F9602BD8274393684F044444444810A2D068064
S12382800A8B4120028B30BD829F3236840F810A2D06800A8B4120028B30BD829F3239F61E
S12382A0102E2AFBB7102F39860DBD829F860ABD829F39860DBD829F860ABD829F860ABDE4
S12382C0829F39A60081FF2706BD829F0820F4390FDF058640B71020B71023B710220E3900
S12382E0DE07270309DF07DE09270309DF098640B710253BB6102EB6102F970086FF970BE6
S12383003BDC05F31018FD1018CE10001D23BF3B4120203D3E2053484F5720504F52542003
S12383204120535441545553FF4220203D3E20434C45415220504F52542042204F55545042
S1238340555453FF4320203D3E2053484F5720504F5254204320535441545553FF44202070
S12383603D3E2053484F5720504F5254204420535441545553FF5220203D3E2053484F57E3
S1238380205245414C2D54494D4520414E414C4F472056414C554553FF5320203D3E204208
S12383A045455020535045414B45522028434F4E4E45435420544F2050413629FF302054EC
S12383C04F2037203D3E20544F47474C45205448452053454C4543544544204220504F5299
S12383E054204C494E45FF3FFF2020545552424F20414441505431314332344458204445FA
S12384004D4F2050524F4752414D204D454E55FF5F5F5F5F5F5F5F5F5F5F5F5F5F5F5F5F40
S12384205F5F5F5F5F5F5F5F5F5F5F5F5F5F5F5F5F5F5F5F5F5F5F5F5FFF4144303DFF41C0
S123844044313DFF4144323DFF4144333DFF4144343DFF4144353DFF4144363DFF414437E2
S12384603DFF504F5254413DFF504F5254433DFF504F5254443DFF504F5254204220434C1B
S11784804541524544FF3E3E3E204245455021203C3C3CFF9A
S123FFD682F480008000800080008000800080008301800080008000800082E0800080002B
S10DFFF6800080008000800080007D
S9030000FC
